:100000000C9461000C9473000C9473000C947300B6
:100010000C9473000C9473000C9473000C94730094
:100020000C9473000C9473000C9473000C94730084
:100030000C9473000C9473000C9473000C94730074
:100040000C9475000C9473000C9473000C94730062
:100050000C9473000C9473000C9473000C94730054
:100060000C9473000C94730000000000250028001D
:100070002B0000000000240027002A0000000000E0
:1000800023002600290004040404040404040202DA
:100090000202020203030303030301020408102007
:1000A0004080010204081020010204081020000012
:1000B0000008000201000003040700000000000027
:1000C000000011241FBECFEFD8E0DEBFCDBF21E07E
:1000D000A0E0B1E001C01D92A930B207E1F70E9493
:1000E000BF000C946E010C9400001F920F920FB68B
:1000F0000F9211242F933F938F939F93AF93BF93AE
:100100008091050190910601A0910701B09108012D
:100110003091040123E0230F2D3758F50196A11DDE
:10012000B11D209304018093050190930601A093D3
:100130000701B09308018091000190910101A09105
:100140000201B09103010196A11DB11D8093000130
:1001500090930101A0930201B0930301BF91AF916D
:100160009F918F913F912F910F900FBE0F901F90F5
:10017000189526E8230F0296A11DB11DD2CF7894C1
:1001800084B5826084BD84B5816084BD85B582609C
:1001900085BD85B5816085BD80916E00816080934D
:1001A0006E001092810080918100826080938100B6
:1001B00080918100816080938100809180008160C6
:1001C000809380008091B10084608093B100809121
:1001D000B00081608093B00080917A008460809349
:1001E0007A0080917A00826080937A0080917A0010
:1001F000816080937A0080917A00806880937A0091
:100200001092C100CCE9D0E0FE01249108E810E092
:10021000F80184918823C9F090E0880F991FFC01B0
:10022000EE58FF4FA591B491FC01E859FF4F45915D
:1002300054913FB7F8949C91822F809598239C937A
:10024000FA019081892380833FBF90EBE92E90E0F3
:10025000F92E20E0C22E20E0D22EF7018491FE017B
:100260009491F8019491992391F0882339F0833087
:10027000F1F098F4813009F1823019F1E92FF0E0C2
:10028000EE0FFF1FE458FF4FA591B4918C91C1145C
:10029000D10419F30E940000E0CF8730A9F0883024
:1002A000C9F0843059F7809180008F7D03C0809120
:1002B00080008F7780938000E1CF84B58F7784BDF5
:1002C000DDCF84B58F7DFBCF8091B0008F77809399
:1002D000B000D4CF8091B0008F7DF9CFF894FFCFDC
:00000001FF
